S1230220C908F10FBD0281BD09EB09EBBD0275FE020130270C05050516068B052208380847
S1230240C908F10FBD0281BD0293C602BD0275FE022AFF0228BD02ADBD028D270C81012754
S12302600B8102270A810327097E03607E038D7E03BA7E03E18609CEFFFF0926FD4A26F78D
S1230280398605CEFFFF0926FD4A26F7398603BD049D39863FB7022C8672B7022DCE04EB99
S12302A0FF022E8639B70230BD022C8339863FFE0228A700081781012E0586717E02C18696
S12302C072A70008FF022808088683A700088639A70008FF0223FE0228B60223A70008B60E
S12302E00224A700FE0223FF022839FE0237FF0226B60231BD049DBD044E39FE023BFF027F
S123030026B60233BD049DBD044E39FE0239FF0226B60232BD049DBD044E39FE023DFF02F4
S123032026B60234BD049DBD044E39FE023FFF0226B60235BD049DBD044E39863EFE02281C
S1230340A70008A70008A70008A70008A70008FF02283986FFFE0228A700BD09EB7E040B3A
S1230360BD02EBBD02FBBD030BBD033BBD02EBBD030BBD031BBD032BBD02EBBD030BBD03DF
S12303803BBD02FBBD02FBBD030B7E0353BD030BBD032BBD02EBBD030BBD033BBD02EBBD7E
S12303A002FBBD030BBD032BBD02EBBD030BBD033BBD02FBBD030B7E0353BD02EBBD02FB59
S12303C0BD030BBD033BBD032BBD02EBBD02FBBD030BBD033BBD02EBBD030BBD031B7E036D
S12303E053BD02EBBD02FBBD030BBD031BBD033BBD02EBBD02FBBD030BBD033BBD032BBDCF
S123040002EBBD02FBBD030B7E0353BD02818601BD049D27037E024AFE022AFF0228B6026E
S123042036BD049DB7022516BD02ADFE0241FF0226B60225BD044E86FFFE0228A700BD0956
S1230440EBB6022581012E03BD047F7E024A48BB0227B702248600B90226B70223FE0223A4
S1230460EE00BF022135FE02283281FF2705A7000820F6863EA70008FF0228BE0221393FB3
S12304808101270BD3D40FD3D01ED3D40F8339C3F000C30856C3F0498339494949B7049CFD
S12304A00E86AFB7C300B60EFCB7049A0FB6C300B7049BC6080CB6049A494949498402B7F9
S12304C00223B6049B84020CB8022327010D79049B79049A5A26DEB6049B0DB2049C250391
S12304E07E04DA0CB9049C4C3904EB150009293F2D0B09183F0D1523373F2B3C1F23082910
S12305002A3F223637373F1F32230C3F253537012A2B3C2903FF051A051E062129FF383261
S123052023FF0572057A05800587058F0596059B05A105A905F405FA05FF0606060D05B19A
S123054005BC05C105C905D005D605E005E705EE0614061A06210627062B0632063A064051
S12305600646064B0655065D066706700677067F06861B0B091E02000DFF0E0B092A3AFFCB
S12305800C0B091F2A29FF1F150018000D2AFF1E2B15000929FF1E152B19FF1F32310C3A77
S12305A0FF1E02180B190B2AFF192D1500210A2AFF2A2D080009182308292AFF1E3D310D63
S12305C0FF192B0B0C1F270DFF2D0B091F2529FF0E18363737FF0E0B091834372D0B14FF05
S12305E00E2B35190A0DFF19343418181EFF1E2E000C25FF2D2308292AFF19373718FF1FA9
S1230600252B0B0A14FF2D0B090D2A3AFF1E2E2516181EFF1D3D180A14FF1D2B131F2A2995
S1230620FF1C2B3C290DFF183D14FF18180621292AFF180B141C3A0B14FF180B0C251EFFD2
S12306401F2A0B0918FF1F0C3D18FF1F2515232B19180B14FF392B15230E0B14FF0F3A0C90
S12306600B091829230DFF2D32310D1E3A0B14FF2D0B09393A1EFF2D15000923181EFF0E5D
S1230680182F001919FF29233214FF06ED06F606FB07010706070C07110715071E072307AB
S12306A02C07330739073F07440749075007580774075D07640769076F0799079F07AA07CB
S12306C0AF07B4077B07820788079307BA07C007C507CE07D407DB07E107EC07F607FD08AE
S12306E004080A0B0F0816081F082508322D15232A3A1D3D18FF2B0B0F3AFF0E2B3C2912B2
S1230700FF0C37370DFF2B0621290DFF2D270D1EFF1F3C29FF0C34342B0D0B0914FF1F0DC9
S12307202628FF1F23320D1F02002AFF181806212919FF251500290DFF112F1E3537FF18B5
S12307403C211DFF1E3D310DFF1C180B092A3AFF1D34342B001F2AFF1B0B0918FF0C00028D
S12307601E3537FF1F23320DFF1C1820211EFF0E3A2B1EFF191815232D1EFF1D3C291818E5
S12307801EFF1D18152D3AFF1D1500212B1D18150029FF1D0200383AFF0E2B161619FF0E7D
S12307A032312A3A1D18150029FF0E161611FF1E363737FF1E32311F2AFF1C2B2F001FFF94
S12307C01B200612FF0C15232D0D2A0A0DFF0D2308292AFF2515230D1E1EFF110621291E57
S12307E0FF1F0D35371D1806212919FF1F0800291801000D1FFF1F15232D0D1EFF1F191532
S1230800000929FF1106212925FF1F3A3A1DFF3932310D1E3AFF0F1521231802002AFF2D97
S123082015232A3AFF2D15000929181E1D18152D3AFF2D0621290FFF085208590860086C9D
S12308400877088208890890089808A308AC08B808BE11062129191FFF1E2B271D2A1FFF70
S12308601B2F00123F1F2A1523251EFF1B2E01123E1D3D180A0DFF1B2E01123F252E001FE7
S12308801EFF1F183C29251FFF192B3C29251FFF1D1832312A3A1FFF1B2E01123F2B0B126F
S12308A00A0DFF27123F1D3D180A14FF27123F2A2B0B0919180B14FF0C3A0C3A1FFF271204
S12308C03F1D1835372A0B14FF08D508D908DD08E108E708EC3D230DFF27090DFF33230F70
S12308E0FF32310D1E3AFF26350F3AFF0D21092BFF08FD09210947096F09AF09CF0D15235E
S12309002A3F0621293F1E2B150009293F150009293F0B090D3F3832233F1B2308371F3F7F
S1230920FF382E002A3F2D32310D3F0C062129191F3F0C3C293F2D15230D2A3F2A37373FD4
S12309401E27000D1F3FFF382E002A3F0B0A123F2D32310D3F33230F3F0C2315213F1D204E
S123096009290F342B0B092A3F2D32310D12FF27091D3F223637373F393D2A3F382F002AA7
S12309803F2D32310D3F2D3223123F1C16161E3F2D0621292A3F2A0B09183F223637373F40
S12309A01B21092B3F38090A1F3F2D32310DFF382E002A3F2D32310D3F0B0A123F252B0AD4
S12309C0092A293F2B35370C2F000D2A0A19FF382E002A3F2D32310D3F0C062129191F3FCF
S10F09E00C3C293F192B15000929FF00CD
S9030000FC
